:020000040000FA
:02000000872D4A
:08000800200023309500A10A3D
:10001000053021020318A1012014A20F1228A30FFA
:100020001228A0144C08003E031930283D1C2E282D
:1000300021000F308C0020008C018C161B22013017
:10004000252200001E30A4008C12073025228C16B9
:1000500006302522A40B24288C1240281B2231288C
:1000600010223630A5000830FF00B120B720C5208F
:10007000142221080B00432859286F2885289B2823
:100080008C010B110900FF1415082B02031C7F15AE
:1000900015082902031C7F1615082A02031CFF16E7
:1000A00021007F088C00200001308C00A50B432824
:1000B000402815082802031C7F1415082602031C7B
:1000C0007F1515082702031C7F16FF1621007F08E5
:1000D0008C00200002308C00A50B592840287F148A
:1000E00015082D02031CFF1415082E02031C7F1691
:1000F00015082C02031CFF1621007F088C0020002D
:1001000004308C00A50B6F28402815082F02031C13
:10011000FF1415083002031C7F147F1515083102E7
:10012000031CFF1621007F088C00200010308C007B
:10013000A50B8528402815083402031CFF14150858
:100140003202031C7F1415083302031C7F157F162F
:1001500021007F088C00200020308C00A50B9B28FC
:1001600040280310350DBE00BE20C100080003105A
:10017000350D013EBE00BE20C200080080308A005E
:100180003E08C93E03188A0A820041088A004208D4
:100190008200813409348134143481341C34813434
:1001A000243481342C348134343481343C348134EB
:1001B000483481344C348134583481345C34813453
:1001C000683481346C348134783481347C348134C3
:1001D000883481348C348134983481349C34813433
:1001E000A8348134AC348134B8348134BC348134A3
:1001F000C8348134CC348134D8348134DC34813413
:10020000E8348134EC348134F8348134FC34823481
:1002100008343C103030C000371811290630B500C2
:100220000A2A0130B5000A2A371819290030B5000A
:100230000A2A0230B5000A2A371821290030B500F1
:100240000A2A0330B5000A2A371829290430B500D4
:100250000A2A0330B5000A2A371831290030B500C0
:100260000A2A0530B5000A2A371839290730B5009F
:100270000A2A0030B5000A2A3718462900304007FC
:1002800003194429C00B0A2A3C140A2AB5010A2A78
:100290003708BB00B50A0A2A3B083706031D522956
:1002A000B5010A2A37183A10371C3A14B50A0A2A37
:1002B0003708BB00B50A0A2A3B083706031D622926
:1002C000B5010A2A37183912371C3916B50A0A2A15
:1002D0003708BB00B50A0A2A3B083706031D7229F6
:1002E000B5010A2A3718B911371CB915B50A0A2AF7
:1002F0003708BB00B50A0A2A3B083706031D8229C6
:10030000B5010A2A37183911371C3915B50A0A2AD6
:100310003708BB00B50A0A2A3B083706031D922995
:10032000B5010A2A3718B910371CB914B50A0A2AB8
:100330003708BB00B50A0A2A3B083706031DA22965
:10034000B5010A2A37183910371C3914B50A0A2A98
:100350003708BB00B50A0A2A3B083706031DB22935
:10036000B5010A2A3718B812371CB816B50A0A2A76
:100370003708BB00B50A0A2A3B083706031DC22905
:10038000B5010A2A37183812371C3816B50A0A2A56
:100390003708BB00B50A0A2A3B083706031DD229D5
:1003A000B5010A2A3718B811371CB815B50A0A2A38
:1003B0003708BB00B50A0A2A3B083706031DE229A5
:1003C000B5010A2A37183811371C3815B50A0A2A18
:1003D0003708BB00B50A0A2A3B083706031DF22975
:1003E000B5010A2A3718B810371CB814B50A0A2AFA
:1003F0003708BB00B50A0A2A3B083706031D022A44
:10040000B5010A2A37183810371C3814B50A0A2AD9
:10041000B5013F1408003C10BC108C1E3C140800B1
:1004200037108C193714080036083502031C1A2AB5
:100430003508B60008003D10CC030310CB0CCA0CE5
:10044000C90CC80C03183D140800C300C30B262AAE
:100450000800C901CA01CB01A030C800C609461C6A
:1004600049144618C914441E4915441AC915C41D17
:100470004916C419C916441D49174419C917C41C83
:100480004A14C418CA14441C4A154418CA15C51E77
:100490004A16C51ACA16451E4A17451ACA17C51D57
:1004A0004B14C519CB14451D4B154519CB15C51C4F
:1004B0004B16C518CB16451C4B174518CB172130CA
:1004C000CC000800CD00CE010830CF000310CD0CC9
:1004D000CE0DCF0B662A4E080800D0000000D00BCE
:1004E0006E2A0800D50A55080D3C0319D501550898
:1004F000C700FE01FD010800D5035508013E031D9C
:10050000842A0C30D500C700FE01FD010800380820
:10051000D500C700F33E031C912A0C30D5025508C4
:100520008A2AFE01FD010800D1002010201C962A15
:10053000D10B952A0800550AD7006222D7005D1812
:10054000D817FF309524D701D801D901013095245F
:10055000080085308700C8308600550AD400160090
:10056000D2001600D300D40BAF2A530886005208DD
:10057000D21787000800F0305202031DC62A530824
:100580007E07DB22FE0FC72AFD0AC72A16000800D5
:1005900023009518C92A8B13151523007E08910096
:1005A0007C089300230055309600AA3096009514DD
:1005B0008B17200008008B1323009518DD2A1511D6
:1005C0002300910023009513151423001308200025
:1005D0008B170800BD30DB22DD000800EA225D1C1D
:1005E000F32A5D10F42A5D14BD30FE005D08FC00A6
:1005F000C8229B229B220800A922FE01FD01BB22EA
:10060000D600D613BB22DC00DC0ABB22DE003F1C76
:10061000252B07303902031D102B8722BF01FC2A2E
:10062000B908031D252B203038020319722221300E
:10063000380203197C22003038020319D5010C302E
:1006400038020319EE22BF01FC2A3C080319372B9C
:100650009B229B223C182F2BBC18332BFC2A722286
:100660009B229B222A2B7C229B229B222A2B02301C
:10067000560203195E2303305602031990230430F7
:10068000560203199F23263056020319FA232730F6
:100690005602031989244C08003E031D5B2BA01C45
:1006A0005B2BA0105D1C562B7222FC2A0730C40065
:1006B0004708C5002922DE0B072BFC2ADF0A5F084A
:1006C000031D672B2330DF00E0096008E10A5F08A3
:1006D00060185F09E200033061020318E101003095
:1006E0006102031D792B6208A600A900AC00AF00CF
:1006F000B20001306102031D832B6208A700AA002B
:10070000AD00B000B30002306102031D8D2B620802
:10071000A800AB00AE00B100B4005C089422080051
:10072000BB22D700BB22D80001305805E300E30A02
:10073000E30DE30D5C089524E30B9A2B0800DF0A18
:100740005F08031DA92B2330DF00E0096008601C4F
:10075000E10A5F0860185F09A600A700A800A900C9
:10076000AA00AB00AC00AD00AE00AF00B000B1001D
:10077000B200B300B4006118A601E118A701611925
:10078000A8016118A901E118AA016119AB0161185A
:10079000AC01E118AD016119AE016118AF01E118BA
:1007A000B0016119B1016118B201E118B301611919
:1007B000B401E119A601E119A701E119A801611A23
:1007C000A901611AAA01611AAB01E11AAC01E11A8F
:1007D000AD01E11AAE01611BAF01611BB001611BEC
:1007E000B101E11BB201E11BB301E11BB4012030F7
:1007F00094220800BB22D700BB22D800BB22E30012
:100800002630840000308500D71B8124D71F852423
:100810002930840000308500571B8124571F852410
:100820002C30840000308500D71A8124D71E8524FF
:100830002F30840000308500571A8124571E8524EC
:100840003230840000308500D7198124D71D8524DB
:10085000273084000030850057198124571D8524D6
:100860002A30840000308500D7188124D71C8524C5
:100870002D3084000030850057188124571C8524B2
:100880003030840000308500D81B8124D81F852497
:100890003330840000308500581B8124581F852484
:1008A0002830840000308500D81A8124D81E852481
:1008B0002B30840000308500581A8124581E85246E
:1008C0002E30840000308500D8198124D81D85245D
:1008D000313084000030850058198124581D85244A
:1008E0003430840000308500D8188124D81C852439
:1008F0005C0894223C18802C3F18802CE30B002CC1
:100900000800800A0319800908008008031D80037D
:100910000800BB22D700BB22D800BB22D900BB22D3
:10092000DA005C08DB00C6240800DB00A601D71B48
:10093000A609A7015719A709A801D81AA809A9014A
:10094000571BA909AA01D718AA09AB01581AAB0964
:10095000AC01D71AAC09AD015718AD09AE01D819D1
:10096000AE09AF01571AAF09B001D81BB009B101E8
:100970005819B109B201D719B209B301581BB3090B
:10098000B401D818B4095B08942208005B08A601DA
:100990004030571BA607A030D71BA607A701403041
:1009A000581AA707A030D81AA707A801403059192C
:1009B000A807A030D919A807A9014030571AA907DC
:1009C000A030D71AA907AA0140305819AA07A030A9
:1009D000D819AA07AB0140305918AB07A030D91875
:1009E000AB07AC0140305719AC07A030D719AC07A2
:1009F000AD0140305818AD07A030D818AD07AE0192
:100A000040305A1BAE07A030DA1BAE07AF014030B2
:100A10005718AF07A030D718AF07B0014030591BA7
:100A2000B007A030D91BB007B10140305A1AB10746
:100A3000A030DA1AB107B2014030581BB207A0301B
:100A4000D81BB207B3014030591AB307A030D91AE6
:100A5000B307B40140305A19B407A030DA19B4070B
:100A60005B0894225B0894225B0894220800003003
:100A7000D7000030D8008030D900FF3095240030F6
:100A8000D900FF3095248030D900FF309524003004
:100A9000D900FF3095248030D900FF3095240230F2
:100AA0003502031C0301D7000030D8000130952423
:100AB0003C0803196B2DB601B5014C08003E031D1F
:100AC000582D3C08D800D70101309524C4010C30C2
:100AD000C5002922582D3F1C4F2DBF01F030D700F3
:100AE000D8017F309524D701D8013F309524F030CC
:100AF000D700D8017F3095243808D7003908D800AE
:100B0000FF309524FF309524B601B5014F2D8C019F
:100B10009501D501CC01BA01B901B801BB01B501FC
:100B2000B601BF01A1010430A100A201A301BC01D3
:100B3000DF01E001E10121007230990023008C0106
:100B40002100823095002100951324008C018C1522
:100B50002000BC018B168B17FF30D700D800D900BE
:100B6000FF309524FF309524D701D801D901FF30FB
:100B70009524FF309524FF309524EA223C08D800C4
:100B8000FF309524FF3095243C1CFC2AEE22372DA3
:100B90008534E234863415348634483486348B34D4
:100BA0008634B8348634F73487341A348734293499
:100BB00087343E3487344534F0340034F034B7346D
:100BC000F034BA34033440341834803400344034C0
:100BD000003420340034103400340834003400343D
:100BE000013400340134003401340434003402345C
:100BF0000034013400340034803400344034003494
:100C00000134003401340034013400342034003421
:100C10001034003408340034043400340234003416
:100C200001340034013400340134263404341034E7
:100C3000FF3400347034FE3402347034FC34063433
:100C40007034F8340E347034F0341E347034E034C0
:100C50003E347034C0347E3470348034FE347034AA
:100C60000134FE3470340334FE3470340734FC3401
:100C700070340F34F83470341F34F03470343F342F
:100C8000E03470347F34C0347034FF3480347034D6
:100C9000033407342034F834003400340034F8349A
:100CA00000340034013400343E3400340034003465
:100CB0003E34003401340034013400340134003453
:100CC0000134003401340034013400340134003480
:100CD00001340034013400343E3400340034003434
:100CE0003E3400340134F834003400340034F83435
:100CF0000034003401340034013400340134003451
:100D0000013400340134003401340034013400343F
:100D1000013400340134263404340E34FF34FE34FC
:100D2000F03400340034F034F8340034F03400345B
:100D30000034F0340734C034F03400340034F0347C
:100D400000343E34F03400340034F034FF34C03426
:100D5000F03400340034F0340734FE34F03400341E
:100D60000034F034F8343E34F03400340034F034DD
:100D7000033430341E3480340034403400342034A2
:100D80000034103400340834003408344034103453
:100D90008034213400344234003484340034043448
:100DA0000034023400340134003400348034003420
:100DB0004034003442340034843401340834023482
:100DC000103404342034003420340034103400341F
:100DD000083400340434003402340834023410344B
:100DE0000434203408344034103480342034033444
:100DF0003034103400342034043410348234083455
:100E00004134043420348234103440340834003403
:100E10000034003408340034103440342034823438
:100E2000413404348234083404341034003420341F
:100E300000340034033430340634803424344034F5
:100E40004234203481341034423420342434403449
:100E500018340334223409348034023440340434E6
:100E60002034083410341034083420341034103452
:100E700020340834403404348034023403342234BF
:100E800002340234AA340534543427342234293449
:100E900040340034003400348034003400340034F2
:100EA000C034003400340034803400340034003462
:100EB0006034003400340034203400340034003412
:100EC0003034003400340034203400340034003432
:100ED0001434003400340034083400340034003456
:100EE0000C3400340034003408340034003400344E
:100EF000053400340034003402340034003400344B
:100F0000033400340034003402340034003400343C
:100F10000134403400340034003480340034003470
:100F20000034C034003400340034803400340034E1
:100F300000344034003400340034303400340034A1
:100F400000343034003400340034303400340034A1
:100F500000340C340034003400340C3400340034D9
:100F600000340C34003400340034033400340034D2
:100F700000340334003400340034033400340034CB
:100F800000340034C034003400340034C034003441
:100F900000340034C03400340034003430340034C1
:100FA0000034003430340034003400343034003441
:100FB000003400340C340034003400340334003482
:100FC000003400340034C034003400340034303491
:080FD0000034003400340C343D
:020000040001F9
:02000E00842943
:02001000FF1ED1
:10E00000270030002D00C034003400340034703458
:10E010000034003400345C340034003400341734ED
:10E020000034003400340534C0340034003401348A
:10E0300040340034003400344034003400340034C0
:10E040000034003400340034C0340034003403346D
:10E050004034003400340D3440340034003435345E
:10E06000003400340034D4340034003400345034EC
:10E0700000340034003440340034003400340034C0
:10E0800030340034003400341C34003400340034A4
:10E0900017340034003400340634C0340034003403
:10E0A000013470340034003400345034003400340F
:10E0B00000341034003400340034003400340034B0
:10E0C00000343034003400340034D03400340034B0
:10E0D00003345034003400340D3440340034003400
:10E0E0003534003400340034143400340034003447
:10E0F000103400340034003400340C340034003464
:10E10000003407340034003400340534C0340034A3
:10E1100000340134B0340034003400345C34003452
:10E120000034003414340034003400340434003437
:10E130000034003400340034003400340C34003433
:10E14000003400343434003400340034D434003427
:10E15000003403345034003400340D34403400347F
:10E160000034053400340034003404340034020038
:0CE1700007000000040007000000000091
:00000001FF
